:1000000011308A00DA290000C135E332EC32F237D0
:10001000ED327439351D20100D0500005034723456
:100020006534763472346134633465346E34FD344F
:100030002034703461346E3465346C3429340D34BA
:100040000A3400347534683465346C3420346E34CA
:1000500061346D34EC34723465346E347934203468
:100060002534313430342E343234663420340D3477
:100070000A340034C135E332EC32F237ED327439F0
:10008000341D20100D05000150346F346434613488
:10009000F83465346E34E93420346E3461347334AA
:1000A00074346134763465346E34ED34203476340F
:1000B000FD349A346B3461343A34203425344C3472
:1000C00064340D340A34003450346F346434613491
:1000D000F83465346E34E93420346E34613473346A
:1000E00074346134763465346E34ED3420346134E4
:1000F0007A3469346D34753474343A3420342534A8
:100100004C3464340D340A340034C135E332EC32FB
:10011000F237ED3274393A10A0060A00C135E332E5
:10012000EC32F237ED327439311D20100D0500012B
:10013000C135E332EC32F237ED327439321D201022
:100140000D0500017A346134643461346E34FD3459
:10015000203461347A3469346D3475347434203425
:100160002534643420340D340A340034A0132008BC
:1001700083168700831287130830F800BF28000019
:10018000F817D028F813D50C03188717031C87130A
:100190007817D0287813F80BC328CE2800008717CB
:1001A0003F308400840BD2280000F81BC228781B43
:1001B000CA280800831603178C170C1400000000CF
:1001C00083120C087F3903191E290313C800031773
:1001D0000D080313C90003170F080313CA004808CA
:1001E000D500B620490803178D0003134A080317EA
:1001F0008F0083168C170C140000000083120C0D66
:100200000E0D7F3903191E290313C80003170D08AB
:100210000313C90003170F080313CA004808D500C9
:10022000B620490803178D0003134A0803178F00EF
:100230008D0A03198F0A0313DA2803170313080022
:100240004008013A03192829033A031931293A29A8
:1002500083168810831288108316081083120814DE
:1002600042298316081083120810831688108312FF
:100270008814422983168810831288108316081068
:100280008312081008000830F80000008711A01140
:1002900020088316870000008312CE0D0712031C6E
:1002A000572920162008831687005B298312201205
:1002B00020088316870000008312A01520088316EB
:1002C00087008312871D6229F80B452900008711DA
:1002D000A011200883168700000083122016200832
:1002E00083168700000000008312A01520088316E3
:1002F00087008312871D7A29F8010000071A7814F5
:100300008711A0112008831687008312071220127C
:100310002008831687008312080020162008831601
:10032000870000008312A0152008831687000000B4
:100330008312071220122008831687000000831200
:100340008711A01120088316870038308312CE0051
:1003500043212A30CE0043210130CE004321201218
:1003600020088316870000008312A015200883163A
:1003700087008312871DBA290000BE2900002016BD
:10038000200883168700000083128A110A16662A45
:1003900040308400831300080319DB290230F80081
:1003A000F701F70BD129F80BD0299730F700F70B9D
:1003B000D729800BCE290800201620088316870035
:1003C00000008312A0152008831687000000831206
:1003D000071220122008831687000000831287115D
:1003E000A0112008831687003C308312CE004321E1
:1003F000CE0143217830CE004321201220088316FD
:10040000870000008312A01520088316870083123E
:10041000871D082A00000C2A0000201620088316D9
:100420008700000006308312C000C8212016200873
:100430008316870000008312A0152008831687000A
:100440000000831207122012200883168700000084
:1004500083128711A0112008831687003C30831275
:10046000CE0043210130CE004321CE014321201292
:1004700020088316870000008312A0152008831629
:1004800087008312871D422A0000462A000020169A
:10049000200883168700000006308312C000C821A0
:1004A000201620088316870000008312A01520085C
:1004B000831687000000831207122012200883167B
:1004C0008700000083128711A0112008831687007F
:1004D0003C308312CE0043210230CE004321CE01B6
:1004E0004321201220088316870000008312A015E4
:1004F0002008831687008312871D7C2A0000802A2B
:1005000000002016200883168700000006308312A2
:10051000C000C8218A110A16692A0830CF0077085E
:10052000D000201620088316870000008312A01533
:100530002008831687008312871D9C2A071A03143C
:10054000071E0310F80D0000A01120088316870075
:1005500083128711CF0B912A20162008831687005B
:1005600000008312071250080319BB2A201220082A
:100570008316870083120000A015200883168700C9
:100580008312871DC12A00008711A011200883163D
:1005900087000000831207122012200883168700AC
:1005A00083120800CA01CB01201620088316870099
:1005B00000008312A0152008831687000000831214
:1005C000071220122008831687000000831287116B
:1005D000A01120088316870038308312CE004321F3
:1005E0004808CE004321201620088316870000000B
:1005F0008312A01520088316870000008312871D30
:10060000FF2A071220122008831687000000831299
:100610008711A01120088316870039308312CE007D
:100620004321F7018D227808CB0020122008831681
:10063000870000008312A01520088316870083120C
:10064000871D202B0000242B000020162008831675
:100650008700000083122016200883168700000000
:100660008312A0152008831687000000831207124A
:100670002012200883168700000083128711A01122
:1006800020088316870038308312CE0043214908A2
:10069000CE00432120162008831687000000831215
:1006A000A01520088316870000008312871D562B93
:1006B000071220122008831687000000831287117A
:1006C000A01120088316870039308312CE00432101
:1006D000F7018D227808CA002012200883168700AF
:1006E00000008312A0152008831687008312871D3F
:1006F000772B00007B2B0000201620088316870034
:1007000000008312CF014B08CE00CF00CE014A0873
:100710004E07F8004F08FA000318FA0A7808CC00D0
:100720007A08CD004D08CF004C08CE00D10104302E
:10073000D0004F0851068039D300CF1FA42BCE091B
:10074000CF09CE0A0319CF0AD11FAB2BD009D1098B
:10075000D00A0319D10AF801F901F701FA01510889
:10076000031DB52B50080319CF2B1030D2000310F6
:10077000CE0DCF0DF70DFA0D51087A02031DC22BD5
:1007800050087702031CCB2B5008F702031CFA0316
:100790005108FA020314F80DF90DD20BB72BD31F31
:1007A000D62BF809F909F80A0319F90A7908CD00D6
:1007B0007808CC004C08F8004D08F90008008E308D
:1007C000F7004D08F8004C08F900FA01CD1FED2B99
:1007D000F809F909F90A0319F80AF808031DFA2BB0
:1007E0007908F800F9010830F702F808031DFA2B20
:1007F000F701032C0310F81B012CF90DF80DF7037A
:10080000FA2BCD1FF81308005D080319C92CE90065
:1008100061080319C92CE902031C132C7F30E90776
:100820000318C92C192C8130E902031CC92C0319A7
:10083000C92C6908F700F801F901FA01E8015E081E
:10084000E700E7175F08E6006008E5001930E900F7
:100850006408E50203183C2C0130E60203183C2C26
:10086000E70203183C2CE80203183C2CE80AE70ACC
:10087000E60A6408E5076E2C6308E6020318572CA5
:100880000130E7020318572CE8020318572CE80A36
:10089000E70A6308E6076408E507031C6E2CE60A0E
:1008A000031D6E2CE70A031D6E2CE80A6E2C6208ED
:1008B0008038E70203186D2C0130E80203186D2C14
:1008C000E80A62088038E7076308E607031C4B2C38
:1008D000E70A031D4B2CE80A4B2C7A14E90B712C08
:1008E0007C2C0310E50DE60DE70DE80D0310FA0D65
:1008F000F90DF80DEA0D282C6A1C842C0310F80C55
:10090000F90CFA0CEA0C872CF7030319C92CEA1B23
:10091000B02C0310E50DE60DE70DE80D6408E502C7
:1009200003189C2C0130E60203189C2CE7020318E4
:100930009C2CE802031CBF2C6308E6020318A72CBA
:100940000130E7020318A72CE802031CBF2C620841
:100950008038E7020318B02C0130E802031CBF2CDA
:10096000FA0A031DBF2CF90A031DBF2CF80A031D48
:10097000BF2CF70A0319C92CF80CF90CFA0C5E0805
:10098000E9006208E906E91FC72CF817CD2CF81317
:10099000CD2CF701F801F901FA0108005A08E1002D
:1009A0005E08E106E11FD92C03110310DA1B0314C2
:1009B0000C2D5A08E1005D08E2005908E202031913
:1009C000E72CE11F0C2D0308013A83000C2D5E0873
:1009D000E2005A08E2020319F32CE11F0C2D030870
:1009E000013A83000C2D5F08E2005B08E202031964
:1009F000FF2CE11F0C2D0308013A83000C2D600829
:100A0000E2005C08E20203190B2DE11F0C2D030824
:100A1000013A83000C2D031008005D0803197D2D99
:100A2000E500610803197D2DE50703181E2D7F30B1
:100A3000E502031C7D2D03197D2D222D8130E50754
:100A400003187D2D6508F700F801F901FA015E0829
:100A5000E900E9175F08E8006008E7001830E500E2
:100A6000E601671C4B2D6408FA07031C3D2DF90AAB
:100A7000031D3D2DF80A0319E6176308F907031C47
:100A8000442DF80A0319E6176208DF00DF175F0834
:100A9000F8070318E617E60DF80CF90CFA0CE90C48
:100AA000E80CE70C0310E50B302D0130F7070318B5
:100AB0007D2DF81B622DE90DFA0DF90DF80DF703E8
:100AC00003197D2DE91F732DFA0A031D732DF90AF1
:100AD000031D732DF80A031D732DF80CF90CFA0C85
:100AE000F70A03197D2D5E08E6006208E606E61F98
:100AF0007B2DF817812DF813812DF701F801F901ED
:100B0000FA01080080308318E206E701E8015E0878
:100B1000E6006208E6065D080319722EE500F7009C
:100B2000610803197B2EE5020319172E031CD52D2E
:100B30006208EB00EB176308EA006408E900E801CB
:100B40000310EB0CEA0CE90CE80CE50B9F2DE61FFB
:100B5000AC2D67148F2E6710651067166030840007
:100B60008313A42E6712E61BBF2D651CCA2DEB0C48
:100B7000EA0CE90CE80CF70A03198A2ECA2DEB1BC4
:100B8000CD2D0310E80DE90DEA0DEB0DF703031968
:100B90008A2EBF2D6717372E67135E08E600E61F03
:100BA000D32DEB17832EEB13832E6108E500F7009E
:100BB0005D08E5025E08EB00EB175F08EA006008DD
:100BC000E900E8010310EB0CEA0CE90CE80CE50B7A
:100BD000E12DE61FEE2DE7148F2EE7106510E716C6
:100BE000643084008313A42EE712E61B012E651CDB
:100BF0000C2EEB0CEA0CE90CE80CF70A03198A2E10
:100C00000C2EEB1B0F2E0310E80DE90DEA0DEB0D7A
:100C1000F70303198A2E012EE717372EE713620810
:100C2000E600E61F152EEB17832EEB13832E6208CA
:100C3000EB00EB176308EA006408E900E61F242EC6
:100C4000EB1367158F2E6711E80165106030840083
:100C50008313A42EE61B4D2E5E08E600651C372E7E
:100C6000EB0CEA0CE90CE80CF70A03198A2EE81FD2
:100C7000482EE90A031D482EEA0A031D482EEB0AF6
:100C8000031D482EEB0CEA0CE90CF70A03198A2E17
:100C9000671BCC2DE71B0E2E6C2E8030EB06EB1F56
:100CA000552E8F2E6208E600622E5E08E600EB08E5
:100CB000031D622EEA08031D622EE908031D622E41
:100CC000F701832EEB1B6C2E0310E80DE90DEA0DE6
:100CD000EB0DF70B622E8A2EE61F702EEB17832E7C
:100CE000EB13832E6108F7006208EB006308EA004B
:100CF0006408E900832E5D08F7005E08EB005F08DA
:100D0000EA006008E9006B08F8006A08F900690861
:100D1000FA00C22EF701F801F901FA01C22EE8012A
:100D2000E909EA09EB09E809E80A031D9D2EE90A29
:100D3000031D9D2EEA0A0319EB0A6718AB2DE7186D
:100D4000ED2D6719232E522E0008E907031CAE2E45
:100D5000EA0A031DAE2EEB0A03196514840300088A
:100D6000EA07031CB62EEB0A031965148403000876
:100D7000801F803AEB0703186514671AB22DE71A33
:100D8000F42D2A2E0800831603178C170C1400006C
:100D9000000083120D080313C90003170F08031383
:100DA000CA0003170C080313D500B620490803171F
:100DB0008D0003134A0803178F008D0A03198F0A49
:100DC0000313C80BC32E0800F701F801F901FA015B
:100DD000DD01DE01DF01E0015C085B045A04590417
:100DE0000319222F2030E1000310D50DD60DD70DA9
:100DF000D80DDD0DDE0DDF0DE00D5C086002031D7A
:100E00000B2F5B085F02031D0B2F5A085E02031DA8
:100E10000B2F59085D02031C1C2F5908DD025A08CC
:100E2000031C5A0FDE025B08031C5B0FDF025C0829
:100E3000031C5C0FE0020314F70DF80DF90DFA0D19
:100E4000E10BF42E5D308400831308008E30F70030
:100E50004008F7024108F9004208F800F917F708BE
:100E600003193D2F0310F908031D392FF808031942
:100E70003D2FF90CF80CF70B322FC11F442FF80946
:100E8000F909F80A0319F90A0800C8010408C7009B
:100E90004810831B4814C11F552FC717471EC70A88
:100EA000C009C109C00A0319C10A410EF038C300C4
:100EB000C307E23EC400323EC60041080F39C407F2
:100EC000C407C607E93EC500C507C507400E0F3970
:100ED000C507C607C50DC60DC609C60D40080F39A2
:100EE000C607C30D0730C2000A30C607C503031C7E
:100EF000752FC507C403031C792FC407C303031C44
:100F00007D2FC307C203031C812F4230840083134B
:100F100007304705471384034705031D962F471ADB
:100F2000840A471A962F2030F700B32F84074630E3
:100F30000402031947170008F700031DA72F471BDA
:100F4000A72F471AC12FC719A72F2030B22FC71FAD
:100F5000AF2F2D30F70084034713C713B32FC715E6
:100F600047123030F707C1010408C0004110831B4D
:100F700041147708D500B620400884008313411837
:100F80008317840A471F972F08004008013A031966
:100F9000CD2F033A0319D62FDF2F83168811831222
:100FA00088118316081183120815E72F831608117C
:100FB000831208118316881183128815E72F831670
:100FC00088118312881183160811831208110800F2
:100FD0003E08F8013D020318F02F3D08F700FC2FF2
:100FE000F7010830BF00BD0DF70D3E08770203186A
:0A0FF000F700F80DBF0BF32F080007
:101000005810D8104B08CF004A08CE004908CD0030
:101010004808CC004B08DC004A08DB004908DA002D
:101020004808D900E001DF01DE01DD018A11CE248C
:101030008A15031C1F2858144D08803ACD00DC0186
:10104000DB01DA017F30D9004F08E0004E08DF00F5
:101050004D08DE004C08DD008A11CE248A15031CE1
:101060004A28E001DF01DE017F30DD004F08E400A7
:101070004E08E3004D08E2004C08E1008A11042408
:101080008A157A08CF007908CE007808CD00770855
:10109000CC00D8140A30E0008930DF003430DE00A4
:1010A0007C30DD004F08E4004E08E3004D08E2000C
:1010B0004C08E1008A110D258A157708D9007808B7
:1010C000DA007908DB007A08DC00E0005B08DF006A
:1010D0005A08DE005908DD004F08E4004E08E3001E
:1010E0004D08E2004C08E1008A110D258A157708A9
:1010F000D9007808DA007908DB007A08DC00831070
:101100005C08E0005B08DF005A08DE005908DD00DB
:101110007C30E4007930E3003530E2008130E100DA
:101120008A1182258A157A08D3007908D2007808B6
:10113000D1007708D0005308E0005208DF005108C2
:10114000DE005008DD004F08E4004E08E3004D08C3
:10115000E2004C08E1008A110D258A157708D900B4
:101160007808DA007908DB007A08DC00E0005B0828
:10117000DF005A08DE005908DD004F08E4004E0881
:10118000E3004D08E2004C08E1008A110D258A15A4
:101190007708D9007808DA007908DB007A08DC00E3
:1011A00083105C08E0005B08DF005A08DE00590885
:1011B000DD003F30E4000230E3003330E2008330F2
:1011C000E1008A1182258A157A08D3007908D200B5
:1011D0007808D1007708D0005308E0005208DF00FB
:1011E0005108DE005008DD004F08E4004E08E3001F
:1011F0004D08E2004C08E1008A110D258A15770898
:10120000D9007808DA007908DB007A08DC00E00011
:101210005B08DF005A08DE005908DD004F08E400D3
:101220004E08E3004D08E2004C08E1008A110D254C
:101230008A157708D9007808DA007908DB007A087F
:10124000DC0083105C08E0005B08DF005A08DE0069
:101250005908DD003330E4008C30E3001E30E2003A
:101260008330E1008A1182258A157A08D300790833
:10127000D2007808D1007708D000E001DF01DE015C
:101280007F30DD004F08E4004E08E3004D08E20027
:101290004C08E1008A110D258A157708D9007808D5
:1012A000DA007908DB007A08DC00E0005B08DF0088
:1012B0005A08DE005908DD004F08E4004E08E3003C
:1012C0004D08E2004C08E1008A110D258A157708C7
:1012D000D9007808DA007908DB007A08DC0083108E
:1012E0005C08E0005B08DF005A08DE005908DD00FA
:1012F0001B30E400E430E3003530E2008230E100EE
:101300008A1182258A157A08D7007908D6007808CC
:10131000D5007708D4005708E0005608DF005508CC
:10132000DE005408DD004F08E4004E08E3004D08DD
:10133000E2004C08E1008A110D258A157708D900D2
:101340007808DA007908DB007A08DC00E0005B0846
:10135000DF005A08DE005908DD004F08E4004E089F
:10136000E3004D08E2004C08E1008A110D258A15C2
:101370007708D9007808DA007908DB007A08DC0001
:1013800083105C08E0005B08DF005A08DE005908A3
:10139000DD00A430E400DB30E3006730E20083309E
:1013A000E1008A1182258A157A08D7007908D600CB
:1013B0007808D5007708D4005708E0005608DF0009
:1013C0005508DE005408DD004F08E4004E08E30035
:1013D0004D08E2004C08E1008A110D258A157708B6
:1013E000D9007808DA007908DB007A08DC00E00030
:1013F0005B08DF005A08DE005908DD004F08E400F2
:101400004E08E3004D08E2004C08E1008A110D256A
:101410008A157708D9007808DA007908DB007A089D
:10142000DC0083105C08E0005B08DF005A08DE0087
:101430005908DD003330E4008C30E3001E30E20058
:101440008330E1008A1182258A157A08D70079084D
:10145000D6007808D5007708D4004F08E0004E0881
:10146000DF004D08DE004C08DD005308E4005208A0
:10147000E3005108E2005008E1008A110D258A15A9
:101480007708D9007808DA007908DB007A08DC00F0
:10149000E0005B08DF005A08DE005908DD0057084D
:1014A000E4005608E3005508E2005408E1008A1100
:1014B00004248A157A08D3007908D2007808D1006C
:1014C0007708D000D81C802A8314DB30E0000F306E
:1014D000DF004930DE007F30DD005308E4005208B1
:1014E000E3005108E2005008E1008A1182258A15C4
:1014F0007A08D3007908D2007808D1007708D000A4
:10150000581C852A5108803AD1005008F70051082C
:10151000F8005208F9005308FA0008000408CD004A
:101520004C08CF000319AF2A4B08E0004A08DF003F
:101530004908DE004808DD00E401E3012030E20054
:101540008230E1008A110D258A157A08CB007908CE
:10155000CA007808C9007708C800CF0B942A4B0846
:10156000D8004A08D7004908D6004808D5005508D1
:10157000B63CD500FA015608D900D6170310D60C90
:10158000D70CD80CFA0CF90CF80CF70CD50BBE2ABA
:10159000D91FD52AF709F809F909FA09F70A031931
:1015A000F80A0319F90A0319FA0A7A08CB0079082C
:1015B000CA007808C9007708C800CB1FEC2ACD0301
:1015C000CD16C809C909CA09CB09C80A0319C90A2D
:1015D0000319CA0A0319CB0A3B30D4009A30D3004E
:1015E000CA30D200D1010A30CF004C080319CD0A0D
:1015F0004B08D8004A08D7004908D6004808D5004B
:101600005408DC005308DB005208DA005108D90006
:101610008A11E4268A150008C800840A0008C90057
:10162000840A0008CA00840A0008CB00FD30840741
:10163000F708031D2E2B4C0A4F0203192E2B4D08C1
:101640000319302B0F394F020319282B0318682B6D
:10165000CD1B682B4D1B302B2030622B2030CD054D
:10166000CD1E402BCD124C08031DCD037708CD00B5
:101670002D30D5008A11B6208A154D08F700CD010E
:101680004C084F02031D502B7708CD002E30D5009B
:101690008A11B6208A154D08F7002030CD0500309C
:1016A0003030CD1E622BCD124C08031DCD037708C0
:1016B000CD002D30D5008A11B6208A154D08F700CF
:1016C000CD013030F7077708D5008A11B6208A158A
:1016D0005408D8005308D7005208D6005108D50046
:1016E000DC01DB01DA010A30D9008A11E4268A150F
:1016F0007A08D4007908D3007808D2007708D1009E
:10170000CF0BF82A8A150A12682D043003178D00B2
:1017100000308F008A110313DA208A150130C800C7
:101720000230C9008A11D2228A157908A2007808ED
:10173000A1000330C8000430C9008A11D2228A15E2
:101740007908A4007808A3000530C8000630C90055
:101750008A11D2228A157908A6007808A5002208E5
:10176000FA002108A21FBD2B2108003CF700FA0156
:101770002208031C220FFA027708A7007A08A800A3
:101780002408FA002308A41FCE2B2308003CF700EE
:10179000FA012408031C240FFA027708C800FA3063
:1017A0004807A9007A08AA000318AA0A2608FA001E
:1017B0002508A61FE42B2508003CF700FA0126089F
:1017C000031C260FFA027708C800FA304807AB005E
:1017D0007A08AC000318AC0A2408CD002308CC001A
:1017E0008A11DF238A157708C8007808C9007908AC
:1017F000CA007A08CB002608CD002508CC008A1143
:10180000DF238A154B08E0004A08DF004908DE00A4
:101810004808DD007A08E4007908E3007808E2006F
:101820007708E1008A1104248A157A08C300790830
:10183000C2007808C1007708C0004308CB00420806
:10184000CA004108C9004008C80000207A08C70043
:101850007908C6007808C5007708C4004708E0008A
:101860004608DF004508DE004408DD00C330E40020
:10187000F530E3004830E2008030E1008A110424B2
:101880008A157708C8007808C9007908CA007A085C
:10189000CB00E0007908DF007808DE007708DD0083
:1018A000E401E3013430E2008630E1008A110D25C5
:1018B0008A157A08C7007908C6007808C500770835
:1018C000C4004408F7004508F8004608F900470836
:1018D000FA00F8134708C7004608C6007808C50094
:1018E0004408C400AA1F772CA81F942C792CA81B8D
:1018F000832C2A082802031C832C031D942C270800
:101900002902031C942CAC1F882CA81F942C8A2C11
:10191000A81BBD2C2C082802031CBD2C031D942CD5
:1019200027082B020318BD2C0E3003178D00003042
:101930008F0083168C170C140000000083128C0893
:101940000319BB2C0D080313C80003170F0803135A
:10195000C90003170C080313D5008A11B6208A1595
:10196000480803178D000313490803178F008D0AD9
:1019700003198F0A992C512D0313A508031DD82C88
:10198000A608031DD82CA41BD32CA408031DCC2C03
:101990002308003C0318D32CC701C6013430C5000E
:1019A0008630C400D72CC701C601C501C401502D23
:1019B000A61B192DA608031DE12C2508003C0318C1
:1019C000192DA41BFE2C8310E001DF013430DE0052
:1019D0008530DD004708E4004608E3004508E200E2
:1019E0004408E1008A1182258A157A08C70079081F
:1019F000C6007808C5007708C400182D8314E001DC
:101A0000DF013430DE008530DD004708E4004608A1
:101A1000E3004508E2004408E1008A1182258A15A6
:101A20007A08C7007908C6007808C5007708C4009E
:101A3000502DA41B362D8314E001DF013430DE006D
:101A40008630DD004708E4004608E3004508E20070
:101A50004408E1008A1182258A157A08C7007908AE
:101A6000C6007808C5007708C400502D8310E00137
:101A7000DF010730DE008730DD004708E40046085C
:101A8000E3004508E2004408E1008A1182258A1536
:101A90007A08C7007908C6007808C5007708C4002E
:101AA000031722308D0000308F000E300313C80062
:101AB0008A11C3268A15093084004708CB004608DE
:101AC000CA004508C9004408C8000230CC008E2A6C
:101AD0002030D5008A11B6208A150D30D5008A1124
:101AE000B6208A150A30D5008A11B6208A15440816
:101AF000F7004508F8004608F9004708FA00080012
:101B00003A3003178D0000308F008A110313DA205A
:101B10008A1585237A08BB007908BA007808B900CD
:101B20007708B8003B08C3003A08C2003908C10072
:101B30003808C0008A1126278A157908BD00780860
:101B4000BC003D08003C0318AF2DFF3A031DAC2D2F
:101B50003C085E3C0318AF2DBD01BC01AF2D3C0815
:101B60003702C000C1013D08031C3D0FC1024108FE
:101B7000BF004008BE00BF08031DC22D3E08023C46
:101B800003181E2E3C083702031DC92DBD0803197A
:101B90001D2EBD08031DD62D37083C020318D62D77
:101BA0000230C0008A1120218A15DB2D0130C000CF
:101BB0008A1120218A153230C0008A11C8218A1565
:101BC0000330C0008A1120218A153230C0008A11EA
:101BD000C8218A1585237A08BB007908BA007808DD
:101BE000B9007708B8003B08C3003A08C2003908BA
:101BF000C1003808C0008A1126278A157908BD005F
:101C00007808BC003D08003C0318102EFF3A031D65
:101C10000D2E3C085E3C0318102EBD01BC01102E99
:101C20003C083702C000C1013D08031C3D0FC10242
:101C30004108BF004008BE00C22DBB2D0330C000CC
:101C40008A1120218A15443003178D0000308F003F
:101C50001A300313C8008A11C3268A151030840075
:101C60003D08C1003C08C0008A1145278A150D3087
:101C7000D5008A11B6208A150A30D5008A11B620FF
:101C80008A158A110A16812ACA01CB01201620085A
:101C90008316870000008312A01520088316870092
:101CA000000083120712201220088316870000000C
:101CB00083128711A0112008831687003C308312FD
:101CC000CE008A1143218A154808CE008A1143218B
:101CD0008A15201620088316870000008312A0159D
:101CE00020088316870000008312871D752E0712B7
:101CF0002012200883168700000083128711A0118C
:101D00002008831687003D308312CE008A114321BC
:101D10008A15F7018A118D228A157808CB002012C6
:101D200020088316870000008312A0152008831660
:101D300087008312871D9A2E00009E2E0000201619
:101D400020088316870000008312201620088316BF
:101D5000870000008312A01520088316870000006A
:101D600083120712201220088316870000008312B6
:101D70008711A0112008831687003C308312CE0003
:101D80008A1143218A154908CE008A1143218A15F8
:101D9000201620088316870000008312A015200853
:101DA0008316870000008312871DD42E071220128D
:101DB000200883168700000083128711A0112008D5
:101DC000831687003D308312CE008A1143218A1585
:101DD000F7018A118D228A157808CA00201220087E
:101DE0008316870000008312A01520088316870041
:101DF0008312871DF92E0000FD2E000020162008FA
:101E00008316870000008312CF014B08CE00CF005D
:101E1000CE014A084E07F8004F08FA000318FA0AE4
:101E20007808CC007A08CD004C08F8004D08F9007D
:101E300008000A168A1100200A128A157A08BB00C7
:101E40007908BA007808B9007708B8003B08C300E1
:101E50003A08C2003908C1003808C0008A11262794
:101E60008A157908BD007808BC003D08003C0318BD
:101E7000432FFF3A031D402F3C085E3C0318432FBD
:101E8000BD01BC01432F3C083702C000C1013D0821
:101E9000031C3D0FC1024108BF004008BE00BF083F
:101EA000031D562F3E08033C0318B62F3C0837028B
:101EB000031D5D2FBD080319B52FBD08031D6A2F33
:101EC00037083C0203186A2F0230C0008A11C52768
:101ED0008A156F2F0130C0008A11C5278A1532304C
:101EE000C0008A11C8218A150330C0008A11C52795
:101EF0008A153230C0008A11C8218A150A168A1143
:101F000000200A128A157A08BB007908BA007808FE
:101F1000B9007708B8003B08C3003A08C200390886
:101F2000C1003808C0008A1126278A157908BD002B
:101F30007808BC003D08003C0318A82FFF3A031D99
:101F4000A52F3C085E3C0318A82FBD01BC01A82F9B
:101F50003C083702C000C1013D08031C3D0FC1020F
:101F60004108BF004008BE00562F4F2F0330C0006D
:101F70008A1120218A15643003178D0000308F00EC
:101F80001B300313C8008A11C3268A151030840041
:101F90003D08C1003C08C0008A1145278A150D3054
:101FA000D5008A11B6208A150A30D5008A11B620CC
:081FB0008A158A110A16872A1E
:102000000330C8000430C9000A128A1544260A1693
:102010008A117908A2007808A1000730C8000830AA
:10202000C9000A128A1544260A168A117908A400E2
:102030007808A3000530C8000630C9000A128A15C6
:1020400044260A168A117908A6007808A5002208F5
:10205000FA002108A21F35282108003CF700FA01E8
:102060002208031C220FFA027708A7007A08A800AA
:102070002408FA002308A41F46282308003CF70080
:10208000FA012408031C240FFA027708A9007A0831
:10209000AA002608FA002508A61F57282508003C94
:1020A000F700FA012608031C260FFA027708AB0096
:1020B0007A08AC002408CD002308CC000A12DF23E4
:1020C0000A167708C8007808C9007908CA007A0893
:1020D000CB002208CD002108CC000A12DF230A160B
:1020E0004B08E0004A08DF004908DE004808DD0030
:1020F0007A08E4007908E3007808E2007708E10054
:102100000A1204240A167A08C3007908C200780863
:10211000C1007708C0004308CB004208CA0041084C
:10212000C9004008C8000A128A1500200A168A1140
:102130007A08C7007908C6007808C5007708C40087
:102140004708E0004608DF004508DE004408DD00DF
:10215000C330E400F530E3004830E2008030E100B5
:102160000A1204240A167708C8007808C9007908FA
:10217000CA007A08CB00E0004A08DF004908DE0008
:102180004808DD00E401E3013430E2008630E1007C
:102190000A120D250A167A08C7007908C6007808C1
:1021A000C5007708C4004408F7004508F800460851
:1021B000F9004708FA00F8134708C7004608C600A8
:1021C0007808C5004408C400A108031D0129A2081D
:1021D000031D0129A41BFA28A408031DF3282308C2
:1021E000003C0318FA28C701C6013430C500853009
:1021F000C4000029C701C6010730C5008730C400EC
:102200005E29A21B2729A208031D0A292108003CD8
:1022100003182729A41F26298314E001DF01343085
:10222000DE008730DD004708E4004608E30045088B
:10223000E2004408E1000A1282250A167A08C70063
:102240007908C6007808C5007708C4005E29A41B79
:1022500044298314E001DF013430DE008630DD00E4
:102260004708E4004608E3004508E2004408E100AE
:102270000A1282250A167A08C7007908C60078086B
:10228000C5007708C4005E298310E001DF01343007
:10229000DE008630DD004708E4004608E30045081C
:1022A000E2004408E1000A1282250A167A08C700F3
:1022B0007908C6007808C5007708C4004408F7000C
:1022C0004508F8004608F9004708FA0008002030E1
:1022D000381E3030B9003708F700B71F7629F709E4
:1022E000F70A7708B7002D30B900B8173708BD00D6
:1022F0006430BE000A12E8270A167708B7003030AB
:102300007807BA003708BD000A30BE000A12E82775
:102310000A1630307707BC0030307807BB00390828
:10232000F700B81D9529B81F3811381AA229B81F0F
:10233000BD293819BD297708BA00B818BD29770812
:10234000BB00BD2930303A02031DBD297708BA0011
:102350002030B900B81DB0293811B814B81FB81012
:1023600030303B02031DBD297708BB002030BA0086
:10237000B81DB029B810B81F3810381DC429390845
:10238000D5000A12B6200A16B81CCB293A08D50087
:102390000A12B6200A16381CD2293B08D5000A12A8
:1023A000B6200A163C08D5000A12B6200A168A1171
:1023B0000A16992A840183131F308305713083160E
:1023C0008F000F088312A013200883168700831242
:1023D0008717831603170908C039890003131F12D2
:1023E0009F1200300317880083128701880189013A
:1023F000FF300313A000831603170908C0398900B2
:1024000003131F129F120030031788008312031357
:102410001F139F1383169F1383121F149412A0126D
:102420002008831687008312201620088316870051
:102430008312A011200883168700013083129400B4
:102440000030831694000108C739083881008312D0
:1024500090010030F8009200003083169200831241
:1024600020152008831687008312970183169B018D
:102470009C0101309D0083120317870188018901A7
:1024800083160908C039890003131F129F122830D0
:10249000031788000908C039890003131F129F120F
:1024A000293003178800853083128D0000308F009B
:1024B0000A120313DA200A160330C0000A12202180
:1024C0000A160A30B500B6000A128D290A160A1239
:1024D000DC290A168E3003178D0000308F000A1297
:1024E0000313DA200A16983003178D0000308F008E
:1024F0000A120313DA200A165A30B7000A128A1594
:10250000802D0A168A11B7010A128A15192F0A1688
:102510008A11A23003178D0000308F000E30031394
:10252000C8000A12C3260A163508B7001F30B800C3
:1025300067292030D5000A12B6200A160D30D500C2
:102540000A12B6200A160A30D5000A12B6200A1658
:102550000830B700FA30C0000A12C8210A16B70BBB
:06256000AA2A732A6300A1
:04400E00F52CFF3F4F
:00000001FF
